:020000020000FC
:10000000B1CDAFC10000000020C0000094C00000CE
:1000100000009EC000000000000000000203040673
:10002000080C10182030406080000406080C1018DE
:100030002030406080A0C00000070F1F3F000D0D62
:1000400004050D050305030302004FB662FD0EC053
:10005000552009F00994C52DC095089483FDC795D6
:10006000C4BDC093A10064604FBE1895C0916400E8
:10007000089483FDC795C4BDC093A1006B7FC09158
:100080006400CF3F09F420C070FF02C082FD05C0AC
:100090004FBE919890989398189575FD0EC065FD88
:1000A0000CC0C091B300C0FD9498C1FD9798C2FDEB
:1000B0009598CAEFC095CA95F1F791989098939842
:1000C0002092A1004FBE189524BCCC27C064C8BFA5
:1000D0006460F6CFC0CF70FFBECF65FDBCCF919AF4
:1000E000BACF70FFB8CF65FDB6CF909AB4CF70FF8E
:1000F000B2CF65FDB0CF939AAECF949A70FFABCFDD
:1001000065FDA9CFC7E0CA95F1F7919AA4CF979A58
:1001100070FFA1CF65FD9FCFC7E0CA95F1F7909A18
:100120009ACF959A70FF97CF65FD95CFC7E0CA9596
:10013000F1F7939A90CF4FB6C9B7CF7EC9BF6E7F04
:10014000CCB5CE0DDDB5DF1DDBBDCABD4FBE1895EC
:100150003FB68F7EABB7A074A2118061A0E0ABBFA9
:10016000A9B7AE7FA9BF7894A0916800AA2341F0F7
:1001700085FD2AC0A0916800AA95A093680024C0BC
:1001800040E050E085FD14C0A0B396FDA095A2FD0F
:100190004FEFA3E096FDA2E0A5BFAA27A064AABFE7
:1001A0008D7FA0B396FDA095A2FD5FEF451741F7A7
:1001B000A8E161FDA093680085FD03C0A8E1A093BC
:1001C000680040939700816085FD0EC0A091690092
:1001D000AA2331F0A0916900AA95A093690004C0F8
:1001E0008061AA27A064AABF80FF37C0A0919700B2
:1001F0004A2F61FF8E7F85FD1CC0A091B600A43000
:10020000C1F4403F08F040EFA42FA295AF704A0F11
:100210005091B800533069F0A695A69550FD01C0E5
:10022000A69552FD03C0A41B4A2F03C04A0F08F431
:100230004FEF40936100A72FA67079F0A0916D0059
:10024000A695A69556E0A50F50916100A50FA09325
:10025000610018F4AFEFA09361004091B600443004
:1002600009F03EC0A0916100A0936300409163003B
:10027000A0919C004A1708F04A2FA0919E004A17AF
:1002800008F04A2F542EA091A200AA2309F422C0FC
:10029000542F5A1B10F4A42F50E0BA2E8894AA1F92
:1002A000AA2EA091A400A095AA22A50E58F0A09174
:1002B000A300A21509F0AA95AA0EA093A30048F0E6
:1002C0004A2D08C0A091A300BA1608F0A395A093E8
:1002D000A3004FEF409364007F7D485F08F0706299
:1002E000A52DA03408F06860A0916000A395A093AC
:1002F000600051F0F894A9B7A160A9BF84FF02C0C3
:10030000A0E4ABBF3FBE1895A0917400A395A09345
:10031000740041E050916800552329F085FF03C027
:100320005A9550936800A0919700A13018F0209240
:100330009A000DC020929B002092A500A0919A00E7
:10034000AF5FA0939A0018F0AFEFA0939A00F894D3
:10035000A9B7A160A9BF84FF02C0A0E4ABBF3FBEA4
:1003600018953FB64CB55DB58F7EABB7A074A211A2
:100370008061A0E0ABBFA9B7AE7FA9BF789481FD33
:1003800023C0A2E096FDA3E0A5BF8260A0B396FDC6
:10039000A095A2FF05C040936500509366003EC142
:1003A000A3E096FDA2E0A5BFAA27A064AABF8D7F07
:1003B00085FF01C026C140E0A0B396FDA095A2FD37
:1003C00020C1409397000FC1A3E096FDA2E0A5BF16
:1003D0008D7F61FF71C0A2E096FDA3E0A5BFAA27B3
:1003E000A064AABF82604093920050939300A090B3
:1003F00090004A19B09091005B09BB24A22C4C38A4
:10040000520518F42092960049C0A091D600AA2364
:1004100059F1483C520528F4A0E1BA2EAAE0AA2ED0
:1004200023C04836A1E05A0728F4A8E0BA2EAFE06E
:10043000AA2E1AC0403DA2E05A0728F4A4E0BA2E22
:10044000AEE1AA2E11C0403AA5E05A0728F4A2E076
:10045000BA2EACE3AA2E08C04839A8E05A0720F407
:10046000A1E0BA2EA8E7AA2EC42EA0919400CA1A21
:10047000D52EA0919500DA0ADD202AF4AFEFC094C2
:10048000D094CA1ADA0A20929600A8E0A210A0E03E
:10049000CA14DA0618F4A1E0A093960040939400E1
:1004A000509395004091920050919300409390009A
:1004B0005093910002E097C0A09165004A1BA09163
:1004C00066005A0B94FD82C093FD80C092FD7CC0F3
:1004D00086FF03C0D52EC42E0CC05695479591FDBE
:1004E00073C05695479590FD6FC0D52EC42ED694F7
:1004F000C79461FD19C0AC2DAC51AD2DA24008F0E0
:1005000005C0DD2089F4AC2DA85C70F4A0916700D3
:10051000A395AA2311F0A0936700AA3008F471C034
:100520002092970081606DC0A0916700AA2319F006
:10053000AA95A0936700A22C5091BC0097FD06C01D
:10054000A090CA00533011F4A090D200AAEFAA0ED6
:10055000A22DA21DCA18DA0A4FB74170533049F4D0
:10056000442321F087FD05C0806803C087FF01C0D8
:100570008F77442359F0533031F4AFEFC094D094C7
:10058000CA1ADA0A03C040E050E020C0533049F4F0
:10059000CC0CDD1CAAE0CA1AD20818F4A0E0CA2EBE
:1005A000D22CAFEFCA16D20418F04FEF50E00EC0B5
:1005B000A091AE00CA9E412D000C441F50E008F0EF
:1005C00012C04FEF50E00FC05695479594FF07C0FB
:1005D000552309F04FEFA42FA6954A0F521D4F3F08
:1005E000520508F04FEF40939700816061FF09C00A
:1005F000AFE1A095A923AB299A2F8F7DBB2009F4E9
:100600008062A8E1A093680085FF03C0AAE0A093E0
:10061000680061FD03C085FD01C08F7E85FD03C0BC
:10062000A6E0A0936900F894A9B7A160A9BF84FFD0
:1006300002C0A0E4ABBF3FBE189511E00AC013E0B2
:1006400008C01AE006C01EE104C014E602C018EC9F
:1006500000C005E1BB27BA95F1F70A95D9F71A95BD
:10066000C1F708952AE338E709C020E33CE806C053
:100670002AE234EB03C025E238EC00C012E095FD1D
:100680009F7D95FF9062BB27979ABA95F1F7909A54
:10069000BA95F1F79098BA95F1F79798BA95F1F75E
:1006A000919AB091AF00BA95F1F79198B7E8BA95E1
:1006B000F1F71A9521F7022FB22FBA95F1F70A95A3
:1006C000D9F73A95D9F6979A0895221B39E0001F79
:1006D0003A9509F40895221F211B18F4210F8894DC
:1006E000F6CF0894F4CF622C722CB0E08894B395C6
:1006F000221F331FE0F7379527958894912E802E7F
:10070000020B130B10F4192D082D10F4889401C05E
:100710000894661C771CBA9571F7172D062D08955D
:10072000322D11232AF43A9500951095031B130BD3
:10073000F894029F712C002D129F912C802C78949C
:10074000780C172D921C292DB4E06B2E2695179549
:1007500007956A94D9F7332321F000951095031B70
:10076000130B08950091B6000430A1F1B0919700E9
:10077000B15008F010C0B0916100B09363002092B6
:100780007F0020928000209281002092820020929F
:1007900083006F7B1FC06090B6006064B091610001
:1007A000B093620008E317EC20917A0030917B004F
:1007B00036952795B62DBA9541F036952795B62DE5
:1007C000BA95BA9511F0369527958DDF00937F0085
:1007D00010938000089500917F00B09162000B1B80
:1007E00010918000120928F40038BFEF1B0740F079
:1007F00009C00F37120508F405C00FE710E002C06A
:1008000000E81FEF00938400109385000895009185
:100810008400B09181000B0F10918500B09182008F
:100820001B1F20E03091850033230AF42A95B091F4
:1008300083002B1F1AF4203F40F00AC02F3008F429
:1008400007C00FEF1FEF2FE003C000E010E020EF24
:1008500030916300B0919C003B1718F4323030F0B7
:1008600009C0B0918500BB235AF004C0B091850047
:10087000BB2332F400938100109382002093830005
:1008800008952091D80000918400000F10918500F8
:10089000111F46DF11232AF40038BFEF1B0740F079
:1008A00009C00F37120508F405C00FE710E002C0B9
:1008B00000E81FEF002352F0B0916200B01B0B2F35
:1008C00018F0013008F00AC001E008C000950F5F81
:1008D000B09162000B0F08F001C00FEF009386008B
:1008E00008952091D900009182001091830018DFB3
:1008F00011232AF40130BFEF1B0740F009C00F3F5E
:10090000120508F405C00FEF10E002C001E01FEF70
:10091000112352F0B0918600B01B0B2F18F001305C
:1009200008F00AC001E008C000950F5FB091860092
:100930000B0F08F001C00FEF0093630008950FEF55
:10094000677F71FD29C072FD09C06860B0917B00AE
:10095000BA3020F0B52DB03408F4677FB091D500DF
:10096000BB23D1F0B0917B00BB23B1F00FEF10910E
:100970007B00ABDEF894B091730072FDB5E00B9F85
:10098000112D002D7894112309F00FEFB0919F00E5
:100990000B1710F400919F0000939E0008950091A2
:1009A0007A0010917B0000541140B0919E0010F429
:1009B000BA9501C0B39511F0B0939E00089500C0A0
:1009C00008952091B700B6B1B6FDFBCF04B115B1C3
:1009D000B6B1BF77B6B9B091AC00B395B093AC00E7
:1009E000B83060F12092AC00B091D400BB2321F16B
:1009F000112329F0B091AD00BF3F61F009C0B09163
:100A0000AD000B1739F020F4BB2321F0BA9502C0DA
:100A1000B395E1F300919C00B093AD00B03050F479
:100A200000ECB03038F400E8B03020F400E4B0302E
:100A300008F400E000939C00777F089510919C00DB
:100A4000B0E11B0F08F41FEF10939C00B091B600AB
:100A5000B43081F000919C00B0916300B01B10F4A1
:100A600000916300B0919E000B1708F00B2F502EE1
:100A700000936400B091AC00B73009F47860089539
:100A800002E3F894B091DA000B9F012D000C001FD7
:100A90007894B0919C000B1710F000919C0000938B
:100AA000610000936300502E0093640000939F0048
:100AB000089520927A00B0EFB0937B000895F894E7
:100AC0000CB51DB52091740078943091750060903C
:100AD00076000093750010937600031B160971FDD4
:100AE00003C076FD81C02BC0709077002093770003
:100AF0002709222311F00FEF1FEF809078009090CC
:100B00007900309378006092790069181619109373
:100B10007C00009175001091760008191909209148
:100B20007A0030917B0036952795020F131F10F441
:100B30000FEF1FEF00937A0010937B0029C02091E4
:100B40007A0030917B003901B4E08B2EB2E09B2E0D
:100B5000343010F08A949A94383010F08A949A9431
:100B6000769467948A94E1F726193709992021F041
:100B7000169507959A94E1F7200F311F20937A007C
:100B800030937B0028F43FEF30937A0030937B0062
:100B9000323008F4706471FF02C0B3E00DC0B09150
:100BA000C60000917100023838F0B395003A08F0A1
:100BB000B395B63008F0B5E09B2EB4E08B2E1091C3
:100BC0007B0000917A0024E0169507952A95E1F7BD
:100BD0000819120928F0B02FB250B12FB20910F441
:100BE00002E010E0980126C020917A0030917B004D
:100BF000390176946794669466946694261932094E
:100C000006950695200F321D20937A0030937B00C5
:100C1000323008F07F7B04E036952795369527958E
:100C200026952695201B10F0223008F422E0890139
:100C30009090C60060FDFECFE0908C00F0908D009B
:100C40006160B9B7B061B9BF380176FD44C0769430
:100C5000679400938C0010938D00B92DB330E1F0B0
:100C6000B0FD04C0060D171D930106C0000F111F33
:100C70000250120922E030E0B92DB33068F0209321
:100C80008E0030938F00009388001093890060924B
:100C90008A0070928B003DC000938E0010938F00ED
:100CA000209388003093890060928A0070928B00B4
:100CB00071FF10C0B0916D00B33060F000918F00F3
:100CC00010917C001595010F28F022F020928E00E3
:100CD00000938F001EC0669400938C00B92DB33032
:100CE00091F0B0FD03C0060D262D03C0000F025089
:100CF00022E0B92DB33038F020938E0000938800A5
:100D000060928A0006C000938E0020938800609253
:100D10008A0000917D0002FD0350013031F495FD01
:100D20000CC0B2E0B06CB7B90BC0023021F4B3E034
:100D3000B06CB7B905C095FDF4CFB4E0B06CB7B9ED
:100D40000091A400000F10F4BBE60B270093A40051
:100D500060FDFECFB2E0B0936E006160B9B7B061E4
:100D6000B9BFB72FB670A1F020917A0030917B0007
:100D700036952795F8940CB51DB5020F131F1BBDB2
:100D80000ABD6160B0E1B8BFB9B7B061B9BF7894CE
:100D90000895606120927E0020E067FD20E206C099
:100DA000606120927E0020E267FD20E0789401E0FF
:100DB00076FD11C0B72FB67009F06F7EB0917B0041
:100DC000B55048F002E0B55020F003E0B55008F00F
:100DD00006E071FD0AE060FD12C0B0917E00BB2309
:100DE00071F071FF08C0B0916D00B33020F0B09188
:100DF0006E00BA9519F4789470615CC0AEDF789497
:100E000000000000F89476FD16C010917B001730AA
:100E100008F017E0B5E01B0F72FD10E183FF110F22
:100E200062FF110F71FD12E8B4B56090A100B61910
:100E300090F2B10B80F2B0B7B77FB0BFB8B1B0B726
:100E4000B860B0BFB0917E00B395B0937E00B8B1EA
:100E500076FD06C0B1E071FDB2E0BA95F1F7B8B128
:100E6000B072B21709F01BC071FF05C003950A30BC
:100E700008F00395B0CF64FF99CF6F7E3CB56DB499
:100E800070907A0080907B00370D681C6BBC3ABD77
:100E90006160B0E1B8BFB9B7B061B9BF87CFB091F9
:100EA0006D00B23008F482CF64FD80CF0A9509F05E
:100EB00092CF7F7E20918E0030918F00F894B0E128
:100EC000B8BF0CB51DB5020F131F1BBD0ABDE090C6
:100ED0008800F09089006160B9B7B061B9BF7894BB
:100EE000B72FB67039F0B0916D0072FFB395B09323
:100EF0006D0009C074FF07C067FD05C064FD03C035
:100F0000BF91BF91E3C4089500E063FF03C064FF95
:100F100001C001E0F89410917100B7E01B9F212DF2
:100F2000102D7894200F26951795269517952695C0
:100F3000179510937100183718F4B8E7B093710043
:100F400000917100B09172000B1720F060629198CF
:100F50009098939860FDFECFE0908A00F0908B000F
:100F60006160B9B7B061B9BF0895B2E095FD07C03F
:100F7000F894B0937D00979A94987894E5C0F8948B
:100F8000B0937D00979A95987894DEC0B3E082FF85
:100F900024C095FD11C002E0F894B0937D00E7E80D
:100FA000F0E00093B3009398959A62FF02C0909A84
:100FB00001C097987894C8C002E0F894B0937D007F
:100FC000E7E8F0E00093B3009198949A62FF02C0C2
:100FD000909A01C097987894B7C095FD0BC0F8948B
:100FE000B0937D00E1E7F0E0939862FF01C0909A32
:100FF0007894AAC0F894B0937D00E1E7F0E091986E
:1010000062FF01C0909A78949FC0B4E095FD07C03C
:10101000F894B0937D00949A9598789495C0F8943C
:10102000B0937D00959A949878948EC0B5E082FF35
:1010300024C095FD11C001E0F894B0937D00EDE768
:10104000F0E00093B3009098979A62FF02C0919AE3
:1010500001C09498789478C004E0F894B0937D002F
:10106000E1E9F0E00093B3009098979A62FF02C024
:10107000939A01C09598789467C095FD0BC0F89439
:10108000B0937D00EBE6F0E0909862FF01C0919A8A
:1010900078945AC0F894B0937D00E7E7F0E0909818
:1010A00062FF01C0939A78944FC0B6E095FD07C0E7
:1010B000F894B0937D00959A9798789445C0F894E9
:1010C000B0937D00949A979878943EC0B1E082FFE7
:1010D00024C095FD11C004E0F894B0937D00E1E9CF
:1010E000F0E00093B3009198949A62FF02C0939A43
:1010F00001C09598789428C001E0F894B0937D00E1
:10110000EDE7F0E00093B3009398959A62FF02C078
:10111000919A01C09498789417C095FD0BC0F894EB
:10112000B0937D00E7E7F0E0919862FF01C0939AE9
:1011300078940AC0F894B0937D00EBE6F0E09398C1
:1011400062FF01C0919A78946F7D08952AE630E09D
:10115000F9012092B300919890989398949A979A55
:10116000959A6B7F0895A4EBB0E009E00D9309E038
:101170000D9304E00D930FEF0D9303E00D930FEF2C
:101180000D930AE00D9303E00D9301E00D9301E050
:101190000D93A0ECB0E001E00D930FEF0D930D93D4
:1011A0000D930D930D9303E00D930FEF0D930FEF40
:1011B0000D930D9305E20D9300ED0D9308E20D9351
:1011C00000E50D9304E00D930FEF0D9302E00D93F6
:1011D00000E00D930AE70D930FEF0D9300E00D93E0
:1011E00001E00D9300E00D9303E00D93089520912D
:1011F000BB008B7F233009F48460B091BC00B33016
:1012000019F09F7DB1FD90629F7BB091BD00B1FD53
:101210009064223011F0886001C0877F08950A959C
:10122000E00FF21DB4910895ECE1F0E00091B400FC
:10123000F6DFB093D800ECE1F0E00091B500EFDF0D
:10124000B093D900EAE2F0E00091BA00E8DFB09391
:10125000DA00B091D0000FEF1CE0B23011F400EAD8
:101260001AE0B33011F402E815E000937200109315
:101270007300E8E3F0E00091D700D1DFB093A20063
:10128000089508952091CA003091CB00B091BC0020
:10129000B33009F43E5097FF02C020E03FEFB32F78
:1012A000B21B6B2EB25810F4B2E86B2E00E003951F
:1012B000609EB12DBD57D8F30093AE00089590689D
:1012C000E1DFC1D920E030E0B0E16B2EB8D9B091B8
:1012D00097002B0F321D6A94C9F7B4E03695279515
:1012E000BA95E1F7822E9F77CDDF0895F894E3E079
:1012F000F0E0B9E0B7BFB491B078C1F3F894A89525
:10130000B1B5B861B1BDB0E0B1BDB4E0BEBFBFE53D
:10131000BDBF1CDFB0E0B8BBB0E1B7BBB0E0B5BB50
:10132000B0E0B4BBB0EBB2BBBBEBB1BB2224A0E0DE
:10133000B0E02D92AA31E9F7A0E6B0E00FEF2D92D0
:101340000A95E9F7B1E0B093A4000DDFF3D2B7E05E
:10135000B06CB7B9B6B1B460B068B6B90091CC00A2
:101360000093AF00B1E0B0936A00F89470D97AD9D5
:101370006AD97BD968D97CD966D9F8940AEF1AEF73
:10138000A0B396FDA095A2FF1FC01A95C9F70A95B4
:10139000B1F7E0E0FCE1B591B43E39F4B591B03E6F
:1013A00021F4B591BF3F09F40CC0E0E0F395F3954B
:1013B000B591B83F49F4B591B43931F4B591BA3A21
:1013C00019F4EE27F695099412DF2EDF5ADF5ADF63
:1013D0000091CC000093AF00B9DEB2E0B3BFB2E041
:1013E000BEBDB2E0B5BDB1E5B8BFB9BFB0B7B77F5C
:1013F000B0BFB8B1B0B7B860B0BF1FD97894DFDA6A
:10140000B3E096FDB2E0B5BFB0E4BBBFBB27B064AC
:10141000BABF8D7F1CD9626033E02CE0B09196009A
:10142000BB2321F42CE03A9509F4A7CF0CD980FF17
:10143000A4CF8E7FB0919700B23078F3B92FBF71EF
:101440000091990000939800B0939900B01729F784
:101450002A9521F76D7FB3E096FDB2E0B5BFBB27BB
:10146000B064BABF8D7FB091D600BB2321F48062F7
:10147000B92FB0709B2F8F7B20926700E6D885FF35
:1014800005C0B0916700BA3008F08064D8D802E097
:1014900085FF01C000E0B0919700B017B8F3F89451
:1014A000E1D8E0D8DFD87894D2D820928700B091E4
:1014B000BC00B33009F474C0C2D8B091C000B130E0
:1014C00008F46EC0B0916A00B13008F469C085FDBF
:1014D00018C0B0919700BF3F08F462C0F894CBD811
:1014E0007894B3D8B0919700B130C0F7F894BAD8D7
:1014F000A8D8B8D87894A9D8B0919700BF3FB0F3D6
:10150000DAC2B3E09B2E9068F894BCDE78949DD844
:10151000F8949F77B7DE80909700B0919700BF371F
:10152000789408F445C089D8F894A5D878949A940A
:1015300051F7C5DEB82DB550B093CB0088D8F894DC
:1015400026D28CD27894BAE09B2E9068F8949ADEDA
:1015500078947BD8F8949F7795DE80909700B0912F
:101560009700BF37789478F768D8F8947BD869D813
:1015700079D878949A9449F7A2DEB82DBB5FB093DE
:10158000CA0065D8F89403D278D278945ED8F894DB
:1015900079DE7894B0919700BF3F08F498CF8BC262
:1015A00000919700B09187000B1710F0009387000F
:1015B0004CD801E0B091BC00B35009F405E0B09103
:1015C0009700B01708F073CFF89455D854D853D873
:1015D00078943DD820926A0020926B0020926C0093
:1015E000B0916B00B395B0936B00BF3F69F5B091BC
:1015F0006C00B395B0936C00B091CE0009E1BA9540
:1016000059F002E3BA9541F00DE7BA9529F00AEFD7
:10161000BA9511F020926C00B0916C00B017A0F058
:10162000B0916C00BA95B0936C00B4EBB0936B00C2
:10163000B091CD00B093AF00F8941DD87894B091DC
:10164000CC00B093AF0001D8FCD7B0916800BB23A9
:1016500019F485FF01C091CE01E085FD01C006E0CF
:10166000B0919700B01708F4BBCFB091BC00B35055
:1016700009F0EBD7B0916800BB2309F47ECEF89453
:1016800065DD209261002092620020926300522C5E
:10169000209264002092A3007894B091B900BB0F0F
:1016A000B093A00020927F002092800020928100C1
:1016B00020928200209283002092AC0060E070E0D3
:1016C00020927100B8E0B093AC007860B6D7B7E074
:1016D00073FDB7E0B06CB7B9B6B1B068B064B6B975
:1016E000B6B1B6FDFDCF04B115B1B6B1BF77B6B98D
:1016F000112309F00FEF0093AD0063D9B8E0B09368
:10170000AC0078608090BB00B2E0B093BB006FDDAE
:101710008092BB00F894BFEFB0939C00B1D9B09118
:101720006100B0939C00B0939D00B0939E007894AC
:10173000B1E0B0936100B09363005B2EB09364009E
:10174000B093A600B0919B00B093A500B091BC00EF
:10175000B33019F49F7D87FD9062716072602092B2
:101760006D00A3DCB3DCA5D9AAD9A3D9A8D9A1D986
:1017700006C0F8943CDD78942092AC00777F10DBB3
:10178000F1D7C2DBF2DB9BD904DB66FD24D876FF00
:10179000D6D876FD04D9B8DBF9DB91D901DB66FD3B
:1017A00036D8B2DB32DC8BD9F4DA66FD6AD8ACDB32
:1017B0003DDC85D9F5DA66FD94D8A6DB76DC7FD9E9
:1017C000E8DAB7E073FDB7E0B06CB7B9B6B1B068AE
:1017D000B064B6B999DB7ADC72D9F3D871FF26C050
:1017E00067FD24C0B0919F00B0939C00B0939D0012
:1017F000B0919B00B093A500B1E0B093A60018E1B2
:101800002CE0B0916D00B11758F07D7F746020938B
:101810006F00B0919F00B0939C00B0939E0006C0F3
:10182000B0919700B13008F0AACF5AC072FF10C033
:1018300067FD0EC0B0916F00BA9511F47B7F99CF10
:10184000B0936F00B0919700B13008F098CF48C0C6
:1018500020927000B0919A000AEFB01708F040C0D3
:1018600085FF04C0B0916800BB23D1F1B091BC00EA
:10187000B33081F495FD03C087FD04C00BC087FF22
:1018800001C008C067FD06C06068B0919F00B093BA
:101890009C008ACF00EF67FF05C0B0919F00B09316
:1018A0009C0000E2B0917B00B01708F468CF67FF9E
:1018B00017C06F779F7D87FD90627460B2E1B0932F
:1018C0006F00B0919F00B0939C0059CFB091700011
:1018D000B395B0937000B0919700BB2309F002C09C
:1018E00020927000F89432DC8090BB00B2E0B0939C
:1018F000BB007DDC8092BB002092610020926200E0
:1019000020926300522C209264002092A0007E7FDF
:10191000789493D61BDCB7E0B06CB7B9B6B1B460BD
:10192000B068B6B985FF05C0B0917000B53008F059
:1019300024CD52CEEDE0F0E023D0053509F01BC0F8
:10194000EEE0F0E01DD00A3A09F015C03AE0A4EB51
:10195000B0E0E3E0F0E014D00D9331963A95D9F77A
:1019600038E1A0ECB0E0EFE0F0E00AD00D93319662
:101970003A95D9F702C0F7DB0AD0E7E2F0E0089524
:10198000E199FECFEEBBFFBBE09A0DB308951ED0E8
:101990003AE0A4EBB0E0E3E0F0E00D910FD0319637
:1019A0003A95D9F738E1A0ECB0E0EFE0F0E00D9126
:1019B00005D031963A95D9F712D00895E199FECF26
:1019C0000DBBEEBBFFBBE29AE19A0895EDE0F0E0BB
:1019D0000FEFF4DFEEE0F0E00FEFF0DF0895EDE061
:1019E000F0E005E5EBDFEEE0F0E00AEAE7DF08957E
:1019F0003091B0000091B100313011F40093B40087
:101A0000323011F40093B500333011F40093B60076
:101A1000343011F40093B800353011F40093BA005B
:101A2000363011F40093C600373011F40093BB0038
:101A3000383011F40093D700393011F40093D000FE
:101A40003A3011F40093BC003B3011F40093BD0018
:101A5000089525E0FCD52A95E9F7089503D605D623
:101A600007D609D6EED5FED500D602D604D6E9D5DE
:101A7000F9D5FBD5FDD5FFD50895FDD5F9D5F5D51B
:101A8000F1D5DFD5F8D5F4D5F0D5ECD5DAD5F3D549
:101A9000EFD5EBD5E7D508958090B0009090B100D8
:101AA000E1D5E0D5DFD5CDD58A94D1F7E4D5C9D538
:101AB0009A94E1F70895F894D1DF7894CADFC9DFEA
:101AC000B1E0B093B000B1E0B093B1002092B200A9
:101AD000F894E2DF7894B5E06B2E70909700B7D55C
:101AE000B09197007B16C9F7B13018F0BF3F40F1B5
:101AF00007C07EDFF8944BDFB1DFB8E0B1BDA9DFEE
:101B00006A9459F7B091B200B395B093B200B33074
:101B100008F4DECF9EDFB091B100B395B093B10071
:101B2000F894B091B000BA95EEE3F0E0EB0FF21D3F
:101B3000049178940395B091B100B01708F4C6CF22
:101B400088DF87DFB091B000B395B093B000B0915B
:101B5000B000BC3008F4B7CF06DBF89418DFB8E06B
:061B6000B1BD77DFC3CB2D
:00000001FF
